S01A000064656D6F70726F675F73746D3332683734332E737265638F
S3150802000000000824550C0208690B02086B0B02084B
S315080200106D0B02086F0B0208710B02080000000044
S31508020020000000000000000000000000730B020838
S31508020030750B020800000000770B0208790B02080C
S31508020040A50C0208A50C0208A50C0208A50C0208B4
S31508020050A50C0208A50C0208A50C0208A50C0208A4
S31508020060A50C0208A50C0208A50C0208A50C020894
S31508020070A50C0208A50C0208A50C0208A50C020884
S31508020080A50C0208A50C0208A50C0208A50C020874
S31508020090A50C0208A50C0208A50C0208A50C020864
S315080200A0A50C0208A50C0208A50C0208A50C020854
S315080200B0A50C0208A50C0208A50C0208A50C020844
S315080200C0A50C0208A50C0208A50C0208A50C020834
S315080200D0A50C0208A50C0208A50C0208A50C020824
S315080200E0A50C0208A50C020800000000A50C0208CF
S315080200F0A50C0208A50C0208A50C0208A50C020804
S31508020100A50C0208A50C0208A50C0208A50C0208F3
S31508020110A50C0208A50C0208A50C0208A50C0208E3
S31508020120A50C0208A50C0208A50C0208A50C0208D3
S31508020130A50C0208A50C0208A50C0208A50C0208C3
S31508020140000000000000000000000000000000009F
S31508020150A50C0208A50C0208A50C0208A50C0208A3
S31508020160A50C0208A50C0208A50C0208A50C020893
S31508020170A50C0208A50C0208A50C0208000000003E
S31508020180A50C0208A50C0208A50C0208A50C020873
S31508020190A50C0208A50C0208A50C0208A50C020863
S315080201A0A50C0208A50C0208A50C0208A50C020853
S315080201B0A50C0208A50C0208A50C0208A50C020843
S315080201C0A50C0208A50C0208A50C0208A50C020833
S315080201D0A50C0208A50C0208A50C0208A50C020823
S315080201E0A50C0208A50C0208A50C0208A50C020813
S315080201F0A50C0208A50C0208A50C0208A50C020803
S31508020200A50C0208A50C0208A50C0208A50C0208F2
S31508020210A50C0208A50C0208A50C0208A50C0208E2
S31508020220A50C0208A50C0208A50C0208000000008D
S31508020230A50C0208A50C020800000000A50C02087D
S31508020240A50C0208A50C0208A50C0208A50C0208B2
S31508020250A50C0208A50C0208A50C0208A50C0208A2
S31508020260A50C0208A50C0208A50C0208A50C020892
S31508020270A50C0208A50C0208A50C0208000000003D
S31508020280A50C0208A50C0208A50C0208000000002D
S3110802029000000000A50C0208EE11AA5599
S3150802029C10B5054C237833B9044B13B10448AFF3A4
S315080202AC00800123237010BD1000002400000000FA
S315080202BC743C020808B5034B1BB103490348AFF358
S315080202CC008008BD0000000014000024743C0208DB
S315080202DC53B94AB9002908BF00281CBF4FF0FF3191
S315080202EC4FF0FF3000F072B9ADF1080C6DE904CE8F
S315080202FC00F006F8DDF804E0DDE9022304B07047E5
S3150802030C2DE9F047089E04468846002B4BD18A42B3
S3150802031C154667D9B2FA82F24AB1C2F1200701FA36
S3150802032C02F320FA07F7954047EA030894404FEA86
S3150802033C154E230CB8FBFEF71FFA85FC0EFB178825
S3150802034C43EA084307FB0CF1994209D9EB1807F162
S3150802035CFF3080F01B81994240F21881023F2B44F0
S3150802036C5B1AA4B2B3FBFEF00EFB103344EA034449
S3150802037C00FB0CFCA44509D92C1900F1FF3380F0BB
S3150802038C0781A44540F2048102382C4440EA07400E
S3150802039CA4EB0C0400271EB1D4400023C6E9004383
S315080203AC3946BDE8F0878B4209D9002E00F0EB805E
S315080203BC0027C6E9000138463946BDE8F087B3FA84
S315080203CC83F7002F47D18B4202D3824200F2FA807E
S315080203DC841A61EB030301209846002EE0D0C6E985
S315080203EC0048DDE702B9FFDEB2FA82F2002A40F0D3
S315080203FC8F80491B4FEA154E1FFA85F80127B1FB68
S3150802040CFEFC230C0EFB1C1143EA014308FB0CF100
S3150802041C994207D9EB180CF1FF3002D2994200F235
S3150802042CCD808446591AA3B2B1FBFEF00EFB10140A
S3150802043C43EA044408FB00F8A04507D92C1900F135
S3150802044CFF3302D2A04500F2B6801846A4EB080484
S3150802045C40EA0C409FE7C7F1200CBB4022FA0CFE7F
S3150802046C4EEA030E01FA07F420FA0CF521FA0CF3FC
S3150802047C4FEA1E482543B3FBF8F92C0C08FB193333
S3150802048C1FFA8EFA44EA034309FB0AF49C4202FA5F
S3150802049C07F200FA07F10BD91EEB030309F1FF3039
S315080204AC80F087809C4240F28480A9F10209734449
S315080204BC1B1BADB2B3FBF8F008FB103345EA034439
S315080204CC00FB0AFAA24508D91EEB040400F1FF3315
S315080204DC6BD2A24569D90238744440EA0940A0FB9A
S315080204EC0289A4EB0A044C45C2464B4654D351D056
S315080204FC002E69D0B1EB0A0564EB030404FA0CFC72
S3150802050CFD40FC404CEA0505C6E90054002747E7BE
S3150802051CC2F1200320FA03F7954001FA02F021FAF8
S3150802052C03F34FEA154E3843010CB3FBFEF71FFAD9
S3150802053C85F80EFB173341EA034107FB08F38B4296
S3150802054C04FA02F407D9691807F1FF3C2FD28B4239
S3150802055C2DD9023F2944CB1A81B2B3FBFEF00EFB0E
S3150802056C103341EA034100FB08F38B4207D9691899
S3150802057C00F1FF3C17D28B4215D902382944C91A05
S3150802058C40EA07473BE73746304609E70746E7E6B8
S3150802059C1846FBE64145ABD2B8EB020A69EB0E02EA
S315080205AC01381346A4E76046E9E7184695E7674615
S315080205BCD1E781467CE702382C4447E7ACF1020CBA
S315080205CC2B442FE7384608E73746E9E6704700BF5B
S315080205DC08B500F077F900F045F900F0B3F808BD54
S315080205EC08B500F049F900F037F908BDF0B4002453
S315080205FC01E00134E4B2112C20D8124D15F814700E
S3150802060C05EB440595F801C007EB0C0606FB00063C
S3150802061C4FF4FA55B5FBF6F506FB05F5B5F5FA5F93
S3150802062CE7D1B5FBF6F60E80013EB6B2B6F5007FFB
S3150802063CDFD2177083F800C0012000E00020F0BC5E
S3150802064C704700BFD83C020808B50948094B036035
S3150802065C4FF46143436000238360C36003610C2239
S3150802066C42618361C3610362836203F092FA08BD35
S3150802067CCC0000240048004070B58CB00025ADF8BB
S3150802068C2E508DF82D500CAB03F8045D0DF12D028E
S3150802069C0DF12E014FF4FA70FFF7A8FF204C214BEF
S315080206AC2360A560E560012626746574A574BDF8F9
S315080206BC2E306361A6619DF82D30E3619DF82C30CE
S315080206CC23626662A662E66226636563A663E563CF
S315080206DC266404236364A564E36425656365A565DA
S315080206ECE56525666566A366204600F089FC0395D2
S315080206FC04950596069640F267630793089309953F
S3150802070C03A9204600F0C6FD00963346022211467E
S3150802071C204600F002FE204600F01BFE0CB070BD0F
S3150802072C2C00002400A0004008B500230122014633
S3150802073C034803F05FF908B1002008BD0120FCE765
S3150802074CCC00002408B5FFF77FFFFFF795FF08BD1D
S3150802075CBFF34F8F0549CA6802F4E062044B134390
S3150802076CCB60BFF34F8F00BFFDE700BF00ED00E083
S3150802077C0400FA0508B5214B1B78B3B92048FFF7D4
S3150802078CD3FF012800D008BD1D4B1B78013BDBB2F9
S3150802079C3F2BF8D800F097F81A4B1860174B012222
S315080207AC1A70194B00221A70EDE7174B1B78013396
S315080207BC13481844FFF7B8FF012813D1124A1378C5
S315080207CC0133DBB213700E4A12789342DBD10B4A11
S315080207DC002111700A4A5278FF2AD4D1022BD2D19F
S315080207ECFFF7B6FF00F06FF8064B1B6864339842A6
S315080207FCC9D9024B00221A70C5E700BF9901002419
S3150802080C580100249C0100249A01002400B58DB0DD
S3150802081C4021104800F096FE10B90DB05DF804FBA5
S3150802082C6B4602AA40210B4800F0AEFD0028F4D113
S3150802083C029A40F267639A42EFD1039B002BECD1E2
S3150802084C9DF816209DF80030FF2BE6D1022AE4D13A
S3150802085CFFF77EFF2C00002408B5FFF78BFFFFF786
S3150802086CD5FF08BD08B500228021024800F068FFB2
S3150802087C08BD00BF0004025810B500F024F80E4B50
S3150802088C1B68C31AB3F5FA7F0CD304460B4B1B78B9
S3150802089C4BB90122094B1A708021094800F050FF06
S315080208AC054B1C6010BD0022044B1A7080210448AB
S315080208BC00F046FFF4E700BFA4010024A0010024BF
S315080208CC00040258704708B500F04AFA08BD000041
S315080208DC014A024B9A6070470000020800ED00E0DC
S315080208EC30B589B0002403940494059406940794AD
S315080208FC1B4BD3F8E02042F08002C3F8E020D3F871
S3150802090CE02002F080020092009AD3F8E02042F02E
S3150802091C0802C3F8E020D3F8E02002F0080201929C
S3150802092C019AD3F8E02042F00202C3F8E020D3F889
S3150802093CE03003F002030293029B0A4D2246802101
S3150802094C284600F0FDFE80230393012304930594A5
S3150802095C069403A9284600F003FE09B030BD00BF71
S3150802096C004402580004025830B5CDB04C2200217E
S3150802097C39A803F070F92022002131A803F06BF98B
S3150802098CBC22002102A803F066F9022000F0DEFE62
S3150802099C00230193254B9A6942F440429A619B695A
S315080209AC03F440430193224BDA6A42F00102DA62FB
S315080209BCDB6A03F001030193019B1C4B9B6913F43D
S315080209CC005FFAD0012339934FF4A0233A930223FA
S315080209DC42934393042544954FF4F07245924693F9
S315080209EC47954893499500244A944B9439A800F0A4
S315080209FCD7FE3F233193032332933394082334933C
S31508020A0C4023359336934FF48062379238932946AE
S31508020A1C31A801F0DFFA48F2020302931D941F94DF
S31508020A2C02A801F073FD4DB030BD00BF0048025854
S31508020A3C0004005808B5FFF74BFF00F057F9FFF70B
S31508020A4C93FFFFF74DFFFFF7C3FDFFF7C9FDFCE761
S31508020A5C82B0074BD3F8F42042F00202C3F8F42012
S31508020A6CD3F8F43003F002030193019B02B07047EA
S31508020A7C0044025800B589B00023039304930593E6
S31508020A8C069307930268154B9A4202D009B05DF891
S31508020A9C04FB134BD3F8EC2042F48072C3F8EC2017
S31508020AACD3F8EC2002F480720192019AD3F8E02072
S31508020ABC42F00202C3F8E020D3F8E03003F0020356
S31508020ACC0293029B4FF44073039302230493092364
S31508020ADC079303A9034800F043FDD7E700A000409B
S31508020AEC004402580004025800B589B00023039347
S31508020AFC04930593069307930268154B9A4202D000
S31508020B0C09B05DF804FB134BD3F8E82042F48022B3
S31508020B1CC3F8E820D3F8E82002F480220192019A5D
S31508020B2CD3F8E02042F00802C3F8E020D3F8E0300C
S31508020B3C03F008030293029B4FF4407303930223B8
S31508020B4C04930723079303A9034800F009FDD7E783
S31508020B5C0048004000440258000C02587047FEE751
S31508020B6CFEE7FEE7FEE770477047704708B500F0E8
S31508020B7CEBF808BD294AD2F8883043F47003C2F858
S31508020B8C8830274B1B6803F00F03062B06D8244A1A
S31508020B9C136823F00F0343F007031360214B1A68FB
S31508020BAC42F001021A6000221A6119681E4A0A40AA
S31508020BBC1A601B4B1B6803F00F03072B06D9184A3E
S31508020BCC136823F00F0343F007031360154B002237
S31508020BDC9A61DA611A62154999621549D9621549F7
S31508020BEC19635A639963DA6319645A64196821F4A6
S31508020BFC802119601A66104B1A68104B1340B3F110
S31508020C0C005F02D20E4B01221A600E4B43F2D2023D
S31508020C1C1A60024B4FF000629A60704700ED00E0D2
S31508020C2C00200052004402587FEDF6EA0002020246
S31508020C3C0000FF01800201010010005C0000FFFFAA
S31508020C4C0881005100400052DFF834D0FFF792FFBA
S31508020C5C002103E00B4B5B58435004310A480B4BFB
S31508020C6C42189A42F6D30A4A02E0002342F8043B97
S31508020C7C084B9A42F9D302F0BFFFFFF7DBFE704727
S31508020C8C00000824443D0208000000241000002439
S31508020C9C10000024AC010024FEE70000104B1B7860
S31508020CAC0BB90120704710B504464FF47A70B0FBA5
S31508020CBCF3F30C4A1068B0FBF3F000F0A1F868B92C
S31508020CCC0F2C01D901200AE0002221464FF0FF30F1
S31508020CDC00F064F8044B1C60002000E0012010BDF3
S31508020CEC08000024000000240C00002410B5032080
S31508020CFC00F042F801F078F80F498B69C3F3032325
S31508020D0C0E4AD35C03F01F03D8408B6903F00F031A
S31508020D1CD35C03F01F0320FA03F3094A1360094B49
S31508020D2C18600020FFF7BAFF10B10124204610BD47
S31508020D3C0446FFF78DFEF9E700440258FC3C02080C
S31508020D4C0400002400000024034B1B78034A116894
S31508020D5C0B441360704700BF08000024A801002446
S31508020D6C014B1868704700BFA8010024014B18688C
S31508020D7C000C70470010005C0649CB6823F4E0634C
S31508020D8C1B041B0C000200F4E0600343024A1A43DC
S31508020D9CCA60704700ED00E00000FA0530B4154B46
S31508020DACDB68C3F30223C3F10704042C28BF04240B
S31508020DBC1D1D062D14D9033B4FF0FF3505FA04F415
S31508020DCC21EA0401994005FA03F322EA03031943BB
S31508020DDC002807DB0901C9B2074B195430BC704706
S31508020DEC0023E9E700F00F000901C9B2034B1954B5
S31508020DFCF4E700BF00ED00E000E400E014ED00E0CB
S31508020E0C0138B0F1807F0AD2064B5860064AF021A7
S31508020E1C82F823100020986007221A607047012076
S31508020E2C704700BF10E000E000ED00E030B4446B00
S31508020E3C0268D2F884106F4B194041EA8401C2F851
S31508020E4C84100268D2F8841021F47F01856B41EA7A
S31508020E5C0541C2F88410826B22440468D4F88810BF
S31508020E6C194041EA8201C4F888100468D4F888103B
S31508020E7C21F4FE01C56B41EA0541C4F88810C16B21
S31508020E8C02EB41020468D4F8A010194041EA820127
S31508020E9CC4F8A0100468D4F8A01021F4FE01056C5D
S31508020EAC41EA0541C4F8A010046C416C01FB042408
S31508020EBC0268D2F8B010194041EA8401C2F8B0109F
S31508020ECC0268D2F8B01021F4FE01856C41EA05419C
S31508020EDCC2F8B010826CC16C01FB02440268D2F8EB
S31508020EECAC10194041EA8401C2F8AC10026D416D8E
S31508020EFC01FB02420468D4F8F010194041EA820157
S31508020F0CC4F8F0100468D4F8F01021F47C11856D3D
S31508020F1C41EA0541C4F8F010816D02EB41020468FE
S31508020F2CD4F8C0100B4043EA8202C4F8C020026807
S31508020F3CD2F8C03023F47C13C16D43EA0143C2F8DC
S31508020F4CC0300268D2F8C03023F07C53016E43EAF3
S31508020F5C0163C2F8C030436B274A1A449200C26630
S31508020F6C836B02EB83030367C16B03EBC103436712
S31508020F7C046C416C01FB04F103EB81038367846CFB
S31508020F8CC16C01FB04F103EB8103C367046D416D6C
S31508020F9C01FB04F103EB8103C0F88030816D03EB8E
S31508020FACC103C0F88430C46D856E05FB04F403EBEB
S31508020FBC8403C0F88830016E01FB05F103EB81034B
S31508020FCCC0F890300D498B420DD9D0F89C3043F0BD
S31508020FDC2003C0F89C30032380F89830012007E0E0
S31508020FEC002342F8043BD0F890309342F8D80020FC
S31508020FFC30BC70470300FFFF002B0010FCD30040E7
S3150802100C30B595B004464C22A04901A802F018FE48
S3150802101C002C00F0388123689D4A934220D094F81C
S3150802102C98300BB32268936923F010039361FFF788
S3150802103C97FE054623689A6912F0080F1AD0FFF72D
S3150802104C8FFE401B0A28F5D9D4F89C3043F00103CD
S3150802105CC4F89C30032384F89830012015B030BDAF
S3150802106C03F580736360DAE784F899302046FFF754
S3150802107C01FDD7E79A6942F001029A61FFF770FE01
S3150802108C054623689A6912F0010F0FD1FFF768FE1D
S3150802109C401B0A28F5D9D4F89C3043F00103C4F84E
S315080210AC9C30032384F898300120D7E79A6942F0DA
S315080210BC02029A61237C012B40D02268936943F081
S315080210CC40039361637C012B3ED02268936923F417
S315080210DC80439361A37C012B3CD02268936943F429
S315080210EC805393612268936923F44073A1680B4376
S315080210FC93612268936923F0A403936122681369A6
S3150802110C23F010031361E368012B29D0002B2CD092
S3150802111C022B00F09B802268936943F0800393614B
S3150802112C2268136943F010031361E368032B1CD17D
S3150802113C2268936943F02003936116E02268936947
S3150802114C23F040039361BDE72268936943F4804315
S3150802115C9361BFE72268936923F480539361C1E7CD
S3150802116C2268936943F004039361A3695A1EE369DF
S3150802117C013B1B0243EA4263226A013A1343626940
S3150802118C013A216843EA0243CB61A368B3F5407F6F
S3150802119C62D0236E33B12268D2F8C030616E0B432B
S315080211ACC2F8C030E36D226ED3420DD02168D1F855
S315080211BCC83023F00703A26E14A800EB820252F879
S315080211CC4C2C1343C1F8C830236C6BB12168D1F887
S315080211DCBC3023F00703626C14A800EB820252F8A7
S315080211EC4C2C1343C1F8BC30A36C73B12168D1F8EB
S315080211FCBC3023F07003E26C14A800EB820252F89E
S3150802120C4C2C43EA0213C1F8BC30236D73B1216826
S3150802121CD1F8BC3023F4E063626D14A800EB8202A9
S3150802122C52F84C2C43EA0223C1F8BC302268184BFC
S3150802123C9A4222D00023C4F89430C4F89C30012375
S3150802124C84F898302046FFF7F1FD07E72268936980
S3150802125C43F02003936188E7A36A013BE26A013AE9
S3150802126C43EA0223226B013A43EA0213626A013AFF
S3150802127C216843EA0243CB608BE76268936823F0E2
S3150802128C03039360D6E70120E8E600BF8C3C02080C
S3150802129C00A0004090F89830013BDBB2012B07D92D
S315080212ACD0F89C3043F00203C0F89C3001207047FA
S315080212BCCB680A68D2B9072B0ED08A68DB0643EAD2
S315080212CC82730A6943EA02434A691343C26E49683E
S315080212DC42F82130002070470A69CB691B0243EA9F
S315080212EC02438A69134343F06053EFE710B40A6961
S315080212FC42EA4372072B0ED08C684B6943EA847315
S3150802130C006F496800EBC10440F831206360002085
S3150802131C5DF8044B70478B69F2E710B490F8984065
S3150802132CE4B2012C09D0D0F89C3043F00403C0F87F
S3150802133C9C3001205DF8044B7047920042EA011179
S3150802134C41EA4303026801990B43C2F88030002034
S3150802135CF0E790F89830DBB2012B07D0D0F89C3026
S3150802136C43F00403C0F89C3001207047022380F82E
S3150802137C98300268936923F0010393610023C0F83D
S3150802138C9C30184670470000F0B490F89840E4B2C6
S3150802139C022C08D0D0F89C3043F00803C0F89C30D5
S315080213AC0120F0BC7047402939D0412964D0046D1C
S315080213BC8C4240F28E80C46F456D01FB05F504EB39
S315080213CC85044FF0000C256805F080455560002D04
S315080213DC40F087802568C5F38A451560256805F0AF
S315080213EC00559560256805F000451561A588D561F7
S315080213FC656805F47025D560656805F48015556130
S3150802140C656805F400159561E57905F07F051562A1
S3150802141C6568ED0F556204F10805002469E0046855
S3150802142CD4F8A05015F4FE0F16D0D4F8A45015F023
S3150802143C7F0F19D0D4F8A45015F0807F01D0D4F8B8
S3150802144CA050D4F8A440C4F3052C446F456C0CFB8D
S3150802145C05F504EB8504B6E7D0F89C3043F0200377
S3150802146CC0F89C3001209CE7D0F89C3043F480737A
S3150802147CC0F89C30012094E70468D4F8B05015F4EF
S3150802148CFE0F16D0D4F8B45015F07F0F19D0D4F835
S3150802149CB45015F0807F01D0D4F8B050D4F8B440CB
S315080214ACC4F3052C846FC56C0CFB05F504EB85049B
S315080214BC89E7D0F89C3043F02003C0F89C30012011
S315080214CC6FE7D0F89C3043F48073C0F89C30012047
S315080214DC67E7D0F89C3043F02003C0F89C30012013
S315080214EC5FE7256825F06045156077E72E5D1E5582
S315080214FC0134D689124FBE5DA642F7D840290BD0C5
S3150802150C41290ED01F2911D80268012303FA01F1C9
S3150802151CC2F89810002044E70368C3F8A8C0002054
S3150802152C3FE70368C3F8B8C000203AE701F01F0189
S3150802153C0268012303FA01F1C2F89C10002030E775
S3150802154C0C3D0208402905D00368D3F8B40000F014
S3150802155C7F0070470368D3F8A40000F07F00704739
S3150802156CF0B583B000233AE0092400E00024B44025
S3150802157C3C4302356E4E46F825406E4C2568D443DC
S3150802158C04EA05064F6817F4803F01D042EA0506BD
S3150802159C684D2E606E6804EA06054F6817F4003F1C
S315080215AC01D042EA0605634E75604FF0B0452D68C8
S315080215BC04EA05064F6817F4801F01D042EA0506AD
S315080215CC4FF0B0452E606D682C404E6816F4001F1D
S315080215DC01D042EA05044FF0B042546001330A685E
S315080215EC32FA03F400F0A28001249C402240F5D082
S315080215FC4D686E1E112D18BF012E01D9122D12D14E
S3150802160C86685F000325BD4026EA0506CD68BD40FF
S3150802161C35438560466826EA04064D68C5F3001408
S3150802162C9C4034434460C6685F000325BD40EC43C6
S3150802163C26408D68BD403543C5604D68122D18BFCE
S3150802164C022D13D1DE08083650F826E003F00705FA
S3150802165C4FEA850C0F2505FA0CF52EEA050E0D69CF
S3150802166C05FA0CF545EA0E0540F82650056825409C
S3150802167C4C6804F00304BC402C4304604C6814F018
S3150802168C805FABD02C4CD4F8F45045F00205C4F864
S3150802169CF450D4F8F44004F002040194019C9D0819
S315080216ACAE1C234C54F8267003F00304A6000F2430
S315080216BCB44027EA0407214CA0423FF457AF04F57D
S315080216CC8064A04222D004F58064A04220D004F59E
S315080216DC8064A0421ED004F58064A0421CD004F596
S315080216EC8064A0421AD004F58064A04218D004F58E
S315080216FC8064A04216D004F58064A04214D004F586
S3150802170C8064A0423FF430AF0A2430E701242EE766
S3150802171C02242CE703242AE7042428E7052426E7CF
S3150802172C062424E7072422E7082420E703B0F0BDA1
S3150802173C0004005880000058004402580000025861
S3150802174C12B909048161704781617047134BDB68D2
S3150802175C13F0040F07D1114BDB6803F0070383421E
S3150802176C1AD00120704710B50C4AD36823F0070328
S3150802177C1843D060FFF7F4FA0446084B5B6813F477
S3150802178C005F07D1FFF7ECFA001BB0F57A7FF4D9A4
S3150802179C012000E0002010BD0020704700480258C6
S315080217AC002800F00C8338B50446036813F0010FC1
S315080217BC25D09D4A136903F03803926A102B15D06B
S315080217CC182B0FD06368B3F5803F3FD0002B53D14B
S315080217DC954B1A6822F480321A601A6822F480220F
S315080217EC1A6038E002F00302022AEBD18E4B1B6810
S315080217FC13F4003F03D06368002B00F0E2822368DF
S3150802180C13F0020F00F08B80874A1369926A13F061
S3150802181C38035AD0182B55D0E368002B00F0C88031
S3150802182C81490A6822F0190213430B60FFF798FAEA
S3150802183C05467D4B1B6813F0040F40F09780FFF7A3
S3150802184C8FFA401B0228F4D90320BFE2764A1368A2
S3150802185C43F48033136063682BB3FFF781FA0546AA
S3150802186C714B1B6813F4003FC9D1FFF779FA401B79
S3150802187C6428F5D90320A9E2B3F5A02F09D06A4B3F
S3150802188C1A6822F480321A601A6822F480221A60C4
S3150802189CE1E7654B1A6842F480221A601A6842F428
S315080218AC80321A60D7E7FFF75BFA05465E4B1B6870
S315080218BC13F4003FA3D0FFF753FA401B6428F5D95B
S315080218CC032083E212F0030FA6D1574B1B6813F0C1
S315080218DC040F03D0E368002B00F07582FFF746FA73
S315080218EC41F20303984212D82269402A07D04E497C
S315080218FC4B6823F47C3343EA02334B600FE04A4AC3
S3150802190C536823F47C3343F40033536007E0464AA6
S3150802191C536823F0FE43216943EA01635360236843
S3150802192C13F0100F00F08A803F4A136903F038034C
S3150802193C926A082B54D0182B4ED0E369002B00F070
S3150802194CBA80394A136843F080031360FFF708FA22
S3150802195C0546354B1B6813F4807F40F08A80FFF7E7
S3150802196CFFF9401B0228F4D903202FE2FFF7FEF9F0
S3150802197C41F20303984212D82269402A07D02A490F
S3150802198C4B6823F47C3343EA02334B60C7E7264A97
S3150802199C536823F47C3343F400335360BFE7224A7B
S315080219AC536823F0FE43216943EA01635360B6E7A1
S315080219BC1D4A136823F001031360FFF7D1F9054694
S315080219CC194B1B6813F0040FA9D0FFF7C9F9401B72
S315080219DC0228F5D90320F9E102F00302012AACD157
S315080219EC114B1B6813F4807F04D0E369802B01D05A
S315080219FC0120EBE1FFF7BAF941F20303984215D835
S31508021A0C226A202A07D008494B6823F0F84343EA8E
S31508021A1C82634B6012E0044A536823F0F84343F09E
S31508021A2C804353600AE000BF004402589A4AD368BE
S31508021A3C23F07C53216A43EA0163D360236813F0CB
S31508021A4C080F60D06369002B49D0934A536F43F051
S31508021A5C01035367FFF784F905468F4B5B6F13F047
S31508021A6C020F50D1FFF77CF9401B0228F5D9032047
S31508021A7CACE1FFF77BF941F20303984212D8226ACA
S31508021A8C202A07D084494B6823F0F84343EA826339
S31508021A9C4B60D3E7804A536823F0F84343F08043FC
S31508021AAC5360CBE77C4AD36823F07C53216A43EA1A
S31508021ABC0163D360C2E7784A136823F08003136084
S31508021ACCFFF74EF90546744B1B6813F4807FB5D0A5
S31508021ADCFFF746F9401B0228F5D9032076E16E4A30
S31508021AEC536F23F001035367FFF73AF905466A4B1E
S31508021AFC5B6F13F0020F06D0FFF732F9401B022870
S31508021B0CF5D9032062E1236813F0200F29D0A369C3
S31508021B1C9BB1614A136843F480531360FFF720F9AB
S31508021B2C05465D4B1B6813F4005F1AD1FFF718F9CB
S31508021B3C401B0228F5D9032048E1574A136823F4B7
S31508021B4C80531360FFF70CF90546534B1B6813F4C5
S31508021B5C005F06D0FFF704F9401B0228F5D90320CB
S31508021B6C34E1236813F0040F21D1636A002B00F0C9
S31508021B7C2C81494A126902F03802182A00F0EE80C2
S31508021B8C022B75D0444A136823F080731360FFF74F
S31508021B9CE7F80446404B1B6813F0007F00F0DC8024
S31508021BACFFF7DEF8001B0228F4D903200EE13B4AA4
S31508021BBC136843F480731360FFF7D2F80546374B64
S31508021BCC1B6813F4807F06D1FFF7CAF8401B6428FA
S31508021BDCF5D90320FAE0A368012B0AD00BBB2E4BCE
S31508021BEC1A6F22F001021A671A6F22F004021A6798
S31508021BFC04E0294A136F43F001031367A36833B34E
S31508021C0CFFF7AEF80546244B1B6F13F0020FACD147
S31508021C1CFFF7A6F8401B41F288339842F3D9032002
S31508021C2CD4E0052B09D01C4B1A6F22F001021A6755
S31508021C3C1A6F22F004021A67E0E7174B1A6F42F082
S31508021C4C04021A671A6F42F001021A67D6E7FFF7FF
S31508021C5C87F80546104B1B6F13F0020F85D0FFF75A
S31508021C6C7FF8401B41F288339842F3D90320ADE042
S31508021C7C094A136823F080731360FFF771F8054657
S31508021C8C054B1B6813F0007F0AD0FFF769F8401B57
S31508021C9C0228F5D9032099E0004402580048025854
S31508021CAC4E4B996A4E4A0A40A16AE06A41EA001109
S31508021CBC0A439A62226B013AC2F30802616B013932
S31508021CCC490289B20A43A16B0139090401F4FE01DE
S31508021CDC0A43E16B0139090601F0FE410A431A630C
S31508021CECDA6A22F00102DA62596B3E4A0A40A16CA0
S31508021CFC42EAC1025A63DA6A22F00C02216C0A43DE
S31508021D0CDA62DA6A22F00202616C0A43DA62DA6A87
S31508021D1C42F48032DA62DA6A42F40032DA62DA6A57
S31508021D2C42F48022DA62DA6A42F00102DA621A684C
S31508021D3C42F080721A60FFF713F80446274B1B68A9
S31508021D4C13F0007F06D1FFF70BF8001B0228F5D912
S31508021D5C03203BE0002039E0002037E01F4A916A55
S31508021D6C106B012B33D001F00303A26A934201D004
S31508021D7C01202BE0C1F30511E36A994201D0012037
S31508021D8C24E0C0F30802236B013B9A4201D00120DE
S31508021D9C1CE0C0F34622636B013B9A4201D0012038
S31508021DAC14E0C0F30642A36B013B9A4211D1C0F36D
S31508021DBC0660E36B013B98420DD0012006E0012038
S31508021DCC7047012002E0012000E0002038BD012006
S31508021DDCFCE70120FAE70020F8E700BF00440258A6
S31508021DEC0CFCFFFF0700FFFF724B1B6903F038035D
S31508021DFC102B00F0DB80182B10D00BB16E487047F5
S31508021E0C6C4B1B6813F0200F00F0D280694B1868D4
S31508021E1CC0F3C100694B23FA00F07047654A916A10
S31508021E2C01F00301906AC0F30510D36A03F00103AB
S31508021E3C526BC2F3CC0203FB02F307EE903AF8EEAE
S31508021E4C677A002800F0B580012966D0F9B1022913
S31508021E5C00F08F8007EE100AF8EE476A9FED586A73
S31508021E6C86EE267A534B1B6BC3F3080306EE903A9F
S31508021E7CF8EE666A9FED536A67EE867A76EEA77A6D
S31508021E8CF7EE006A77EEA67A27EE277A61E0494BD7
S31508021E9C1B6813F0200F23D046490A68C2F3C10205
S31508021EAC464BD34007EE103AF8EE476A07EE100A8D
S31508021EBCB8EE476A86EE867A0B6BC3F3080306EE10
S31508021ECC903AF8EE666A9FED3F6A67EE867A76EE88
S31508021EDCA77AF7EE006A77EEA67A27EE277A38E023
S31508021EEC07EE100AF8EE476A9FED376A86EE267AEF
S31508021EFC304B1B6BC3F3080306EE903AF8EE666A90
S31508021F0C9FED306A67EE867A76EEA77AF7EE006A66
S31508021F1C77EEA67A27EE277A1BE007EE100AF8EE7A
S31508021F2C476A9FED276A86EE267A224B1B6BC3F30A
S31508021F3C080306EE903AF8EE666A9FED226A67EE99
S31508021F4C867A76EEA77AF7EE006A77EEA67A27EE07
S31508021F5C277A184B1B6BC3F34623013307EE903AC9
S31508021F6CF8EE677AC7EE276AFCEEE67A17EE900A5F
S31508021F7C704707EE100AF8EE476A9FED146A86EE6A
S31508021F8C267A0C4B1B6BC3F3080306EE903AF8EE53
S31508021F9C666A9FED0C6A67EE867A76EEA77AF7EE94
S31508021FAC006A77EEA67A27EE277AD2E708487047B0
S31508021FBC024870470044025800093D000090D003BD
S31508021FCC0024744A000000390024744C0024F44A94
S31508021FDC00127A00002800F0368103469C4A1268E1
S31508021FEC02F00F028A420CD29948026822F00F02BA
S31508021FFC0A430260026802F00F028A4201D00120EB
S3150802200C704770B51A6812F0040F0CD01869914A09
S3150802201C926902F07002904205D98E4CA26922F09E
S3150802202C70021043A0611A6812F0080F0CD0586996
S3150802203C884AD26902F07002904205D9854CE26947
S3150802204C22F070021043E0611A6812F0100F0CD0DD
S3150802205C9869804AD26902F4E062904205D97D4CAD
S3150802206CE26922F4E0621043E0611A6812F0200F6A
S3150802207C0CD0D869774A126A02F07002904205D9D6
S3150802208C744C226A22F07002104320621A6812F00B
S3150802209C020F0CD0D8686F4A926902F00F0290426E
S315080220AC05D96C4CA26922F00F021043A0611C469A
S315080220BC0D461B6813F0010F41D0664A936923F447
S315080220CC7063A1680B4393616368022B0AD0032BD6
S315080220DC27D0012B2CD05F4A126812F0040F06D1B6
S315080220EC0120AFE0126812F4003F00F0AE805949A5
S315080220FC0A6922F0070213430B61FEF731FE064604
S3150802210C544B1B6903F038036268B3EBC20F16D043
S3150802211CFEF726FE801B41F288339842F0D903203B
S3150802212C90E04C4A126812F0007FE0D1012089E057
S3150802213C484A126812F4807FD9D1012082E02368BA
S3150802214C13F0020F0CD0E268424B9B6903F00F03A3
S3150802215C9A4205D23F498B6923F00F031A438A61C7
S3150802216C3B4B1B6803F00F03AB420CD9384A136876
S3150802217C23F00F032B431360136803F00F03AB42D0
S3150802218C01D001205EE0236813F0040F0CD02269FB
S3150802219C304B9B6903F070039A4205D22D498B6921
S315080221AC23F070031A438A61236813F0080F0CD0C4
S315080221BC6269284BDB6903F070039A4205D22549FA
S315080221CCCB6923F070031A43CA61236813F0100F04
S315080221DC0CD0A2691F4BDB6903F4E0639A4205D261
S315080221EC1C49CB6923F4E0631A43CA61236813F0CA
S315080221FC200F0CD0E269174B1B6A03F070039A4244
S3150802220C05D214490B6A23F070031A430A62FFF7C4
S3150802221CEBFD10498B69C3F303230F4AD35C03F016
S3150802222C1F03D8408B6903F00F03D35C03F01F031B
S3150802223C20FA03F3094A1360094B1860094B18680C
S3150802224CFEF72CFD70BD012070470120FAE700BF8E
S3150802225C0020005200440258FC3C020804000024E8
S3150802226C000000240C00002408B5FFF7BDFD0B4A3C
S3150802227C9369C3F303230A49CB5C03F01F0320FAC1
S3150802228C03F3926902F00F02885C00F01F0023FA2E
S3150802229C00F0044A1060044A136008BD0044025850
S315080222ACFC3C0208040000240000002408B5FFF7D1
S315080222BCDBFF054BDB69C3F30213044AD35C03F059
S315080222CC1F03D84008BD00BF00440258FC3C020854
S315080222DC08B5FFF7C9FF054BDB69C3F30223044AAA
S315080222ECD35C03F01F03D84008BD00BF0044025854
S315080222FCFC3C0208404B9B6A03F00303032B79D080
S3150802230C70B50E4604463C4A136823F08063136084
S3150802231CFEF726FD0546384B1B6813F0006F06D0F0
S3150802232CFEF71EFD401B0228F5D9032070BD324B61
S3150802233C9A6A22F47C32216842EA01329A6262680B
S3150802234C013AC2F30802A1680139490289B20A4361
S3150802235CE1680139090401F4FE010A4321690139CC
S3150802236C090601F0FE410A439A63DA6A22F0C002B0
S3150802237C61690A43DA62DA6A22F02002A1690A431F
S3150802238CDA62DA6A22F01002DA62D96B1B4A0A405E
S3150802239CE16942EAC102DA63DA6A42F01002DA62E7
S315080223ACC6B91A46DB6A43F40023D362124A136887
S315080223BC43F080631360FEF7D3FC04460E4B1B688E
S315080223CC13F0006F14D1FEF7CBFC001B0228F5D9CB
S315080223DC0320ABE7012E05D0074AD36A43F4001350
S315080223ECD362E3E7044AD36A43F48013D362DDE784
S315080223FC00209BE701207047004402580700FFFFA4
S3150802240C404B9B6A03F00303032B79D070B50E4637
S3150802241C04463C4A136823F080531360FEF7A0FC6B
S3150802242C0546384B1B6813F0005F06D0FEF798FC7E
S3150802243C401B0228F5D9032070BD324B9A6A22F04A
S3150802244C7C72216842EA01529A626268013AC2F3C4
S3150802245C0802A1680139490289B20A43E1680139BD
S3150802246C090401F4FE010A4321690139090601F03E
S3150802247CFE410A431A64DA6A22F4406261690A4323
S3150802248CDA62DA6A22F40072A1690A43DA62DA6A51
S3150802249C22F48072DA62596C1B4A0A40E16942EAF2
S315080224ACC1025A64DA6A42F48072DA62C6B91A4608
S315080224BCDB6A43F48003D362124A136843F08053EF
S315080224CC1360FEF74DFC04460E4B1B6813F0005FB7
S315080224DC14D1FEF745FC001B0228F5D90320ABE7FD
S315080224EC012E05D0074AD36A43F08073D362E3E719
S315080224FC044AD36A43F40003D362DDE700209BE760
S3150802250C01207047004402580700FFFFF8B504463D
S3150802251C036813F0006F2BD0436EB3F5801F18D0E7
S3150802252C07D9B3F5001F1DD0B3F5401F2ED10025D0
S3150802253C06E05BBB934AD36A43F40033D3620025A5
S3150802254C904A136D23F44013616E0B4313650026F0
S3150802255C10E002210430FFF7CDFE0546002DEFD020
S3150802256C2E4607E002212430FFF74AFF0546F5E717
S3150802257C00263546236813F4807F17D0636D042B27
S3150802258C32D8DFE803F006242A0B0B00012635465F
S3150802259CF0E77C4AD36A43F40033D3623DBB794AEB
S315080225AC136D23F00703616D0B431365236813F44C
S315080225BC007F33D0A36D802B44D01AD80BB3402B93
S315080225CC1CD10021201DFFF795FE05461EE00021B1
S315080225DC201DFFF78FFE0546E0E7002104F12400D3
S315080225ECFFF70EFF0546D9E701263546DEE72E46E6
S315080225FCDCE7C02B0AD0B3F5807F07D00126354617
S3150802260C0CE0604AD36A43F40033D3620DBB5D4ACD
S3150802261C136D23F4E073A16D0B431365236813F44E
S3150802262C806F2FD0D4F8A430B3F5800F3ED012D8D1
S3150802263CD3B1B3F5001F14D10021201DFFF75AFEA2
S3150802264C054616E0002104F12400FFF7D9FE0546DB
S3150802265CDCE72E46E2E7B3F5C00F0AD0B3F5000F56
S3150802266C07D0012635460DE0464AD36A43F40033B1
S3150802267CD36215BB434A936D23F46003D4F8A410B2
S3150802268C0B439365236813F4006F2FD0D4F8A83044
S3150802269CB3F1007F37D012D8D3B1B3F1807F14D1FE
S315080226AC0021201DFFF726FE054616E0002104F13F
S315080226BC2400FFF7A5FE0546DBE72E46E2E7B3F153
S315080226CC407F0AD0B3F1806F07D0012635460DE05C
S315080226DC2C4AD36A43F40033D362DDB9294A936D83
S315080226EC23F0E063D4F8A8100B439365236813F020
S315080226FC007F2AD0A36C102B12D00DD9202B1DD0FB
S3150802270C302B12D009E0002104F12400FFF778FEE1
S3150802271C0546E2E72E46E9E73BB10126354614E0C3
S3150802272C184AD36A43F40033D3626DB9154AD36C8B
S3150802273C23F03003A16C0B43D36406E00221201D5F
S3150802274CFFF7D8FD0546F0E72E46236813F4805F9B
S3150802275C27D0E36DB3F5005F3ED009D8A3B1B3F524
S3150802276C805F0BD10021201DFFF7C4FD054610E042
S3150802277CB3F5405F0DD0B3F5804F0AD00126354626
S3150802278C0FE000BF00440258934AD36A43F400335D
S3150802279CD36245BB904A136D23F4E043E16D0B43B8
S315080227AC1365236813F4005F33D0236EB3F5003F29
S315080227BC27D01AD83BB1B3F5803F1FD10121201D72
S315080227CCFFF798FD05461DBB834A136D23F4E023D8
S315080227DC216E0B4313651CE0002104F12400FFF75C
S315080227EC0FFE0546D5E72E46DBE7B3F5802FEAD072
S315080227FCB3F5A02FE7D0B3F5403FE4D00126354612
S3150802280C07E0012104F12400FFF7FAFD0546DAE791
S3150802281C2E46236813F4804F2CD0D4F8AC30B3F17F
S3150802282C005F1FD012D83BB1B3F1805F17D10121DB
S3150802283C201DFFF75FFD0546DDB9674A936D23F048
S3150802284CE043D4F8AC100B43936513E0B3F1804F15
S3150802285CF2D0B3F1A04FEFD0B3F1405FECD0012622
S3150802286C354607E0012104F12400FFF7C9FD0546A8
S3150802287CE2E72E46236813F4004F1FD0E36EB3F13A
S3150802288C805F06D0B3F1005F11D03BB10126354605
S3150802289C14E0514AD36A43F40033D3626DB94E4AF3
S315080228AC136D23F04053E16E0B43136506E00121C9
S315080228BC201DFFF71FFD0546F0E72E46236813F089
S315080228CC807F1ED0636C032B17D8DFE803F0070250
S315080228DC1007414AD36A43F40033D36285B93E4A98
S315080228ECD36C23F00303616C0B43D36409E0022116
S315080228FC201DFFF7FFFC0546F0E70126354600E0EA
S3150802290C2E46236813F4800F1FD1236813F0010F88
S3150802291C00F09E80A36F282B00F29680DFE803F066
S3150802292C84949494949494947F9494949494949470
S3150802293C8D94949494949494849494949494949452
S3150802294C84949494949494948400244A136843F437
S3150802295C80731360FEF704FA0746204B1B6813F4C0
S3150802296C807F05D1FEF7FCF9C01B6428F5D903252F
S3150802297C002D50D1184B1B6FD4F8B020534013F4CA
S3150802298C407F0CD0144B1A6F22F44072196F41F423
S3150802299C80311967196F21F4803119671A67D4F8CF
S315080229ACB030B3F5807F1BD0002D36D1D4F8B030B9
S315080229BC03F44072B2F5407F23D0074A136923F415
S315080229CC7C53136104490B6FD4F8B020C2F30B0283
S315080229DC13430B6799E700BF004402580048025894
S315080229ECFEF7BEF90746AC4B1B6F13F0020FDBD191
S315080229FCFEF7B6F9C01B41F288339842F3D9032580
S31508022A0CD2E7A548026922F47C52A44901EA1313B7
S31508022A1C13430361D6E72E4677E72E4675E701215F
S31508022A2C201DFFF767FC05468DB99B4A536D23F0AB
S31508022A3C3803A16F0B4353650AE0012104F1240004
S31508022A4CFFF7DEFC0546EFE70126354600E02E4683
S31508022A5C236813F0020F20D0636F052B19D8DFE811
S31508022A6C03F00803110808080121201DFFF742FC90
S31508022A7C05468DB9884A536D23F00703616F0B43DC
S31508022A8C53650AE0012104F12400FFF7B9FC054657
S31508022A9CEFE70126354600E02E46236813F0040FAD
S31508022AAC22D0D4F89030052B1AD8DFE803F00803A5
S31508022ABC120808080121201DFFF71CFC054695B9CA
S31508022ACC754A936D23F00703D4F890100B4393655C
S31508022ADC0AE0012104F12400FFF792FC0546EEE711
S31508022AEC0126354600E02E46236813F0200F2CD01B
S31508022AFCD4F88C30B3F1005F1FD012D83BB1B3F1C6
S31508022B0C805F17D10021201DFFF7F4FB0546DDB9BE
S31508022B1C614A536D23F0E043D4F88C100B4353658A
S31508022B2C13E0B3F1804FF2D0B3F1A04FEFD0B3F16B
S31508022B3C405FECD00126354607E0022104F1240059
S31508022B4CFFF75EFC0546E2E72E46236813F0400FB4
S31508022B5C2CD0D4F89830B3F5006F1FD012D83BB1ED
S31508022B6CB3F5806F17D10021201DFFF7C3FB05466D
S31508022B7CDDB9494A936D23F4E053D4F898100B4304
S31508022B8C936513E0B3F5805FF2D0B3F5A05FEFD08F
S31508022B9CB3F5406FECD00126354607E0022104F165
S31508022BAC2400FFF72DFC0546E2E72E46236813F0B0
S31508022BBC800F2CD0D4F89C30B3F5804F1FD012D886
S31508022BCC3BB1B3F5005F17D10021201DFFF792FB2D
S31508022BDC0546DDB9304A936D23F46043D4F89C104C
S31508022BEC0B43936513E0B3F5004FF2D0B3F5204FC0
S31508022BFCEFD0B3F5C04FECD00126354607E00221DB
S31508022C0C04F12400FFF7FCFB0546E2E72E4623688F
S31508022C1C13F0080F0CD0D4F88030B3F5805F28D0A7
S31508022C2C1D4A536D23F44053D4F880100B43536555
S31508022C3C236813F0100F0CD0D4F89430B3F5807FB8
S31508022C4C20D0154A936D23F44073D4F894100B4391
S31508022C5C9365236813F4002F39D0D4F8A030B3F552
S31508022C6C803F2CD0B3F5003F1FD0CBB10126354699
S31508022C7C2DE0022104F12400FFF7C2FB0028CFD075
S31508022C8C0126CDE7022104F12400FFF7B9FB00283F
S31508022C9CD7D00126D5E700BF00440258CFFFFF0064
S31508022CAC0021201DFFF726FB05467DB9644A936D64
S31508022CBC23F44033D4F8A0100B43936507E00221A2
S31508022CCC04F12400FFF79CFB0546EEE72E46236823
S31508022CDC13F4802F24D0D4F88430B3F5001F17D000
S31508022CECB3F5401F0AD0B3F5801F02D0012635462C
S31508022CFC16E0534AD36A43F40033D3627DB9504A79
S31508022D0C536D23F44013D4F884100B43536507E030
S31508022D1C012104F12400FFF773FB0546EEE72E4664
S31508022D2C236813F4803F14D0E36C2BB1B3F5803FC0
S31508022D3C23D0012635460CE0414AD36A43F40033C4
S31508022D4CD36205BB3E4AD36C23F48033E16C0B4346
S31508022D5CD364236813F0005F17D1236813F4003F7A
S31508022D6C2DD0E36FB3F5807F1BD017D9B3F5007F4F
S31508022D7C1CD0B3F5407F12D118E00221201DFFF7B3
S31508022D8CB9FA0546DDE72E46E3E7022104F12400EB
S31508022D9CFFF736FB0028E0D00126DEE733B1012621
S31508022DAC0DE0274AD36A43F40033D362002D3DD192
S31508022DBC234A536D23F44073E16F0B43536523681F
S31508022DCC13F4801F06D01E4A136D23F00043216F9D
S31508022DDC0B431365236813F0805F07D0184A1369EF
S31508022DEC23F48043D4F8B4100B431361236813F409
S31508022DFC001F06D0124A136D23F08073A16E0B4383
S31508022E0C1365236813F0804F09D00D4B1A6922F407
S31508022E1C00421A611A69D4F8B8100A431A6123686F
S31508022E2C002B05DB06B101263046F8BD2E46C6E751
S31508022E3C034AD36C23F04053216D0B43D364F1E759
S31508022E4C0044025808B5FFF70FFA054B1B6AC3F381
S31508022E5C0213044AD35C03F01F03D84008BD00BF13
S31508022E6C00440258FC3C020810B478498C6A8A6AF7
S31508022E7CC2F30532CB6AC3F30013C96BC1F3CC0197
S31508022E8C03FB01F3002A00F0DB8004F0030407EECF
S31508022E9C903AF8EE677A012C66D0FCB1022C00F057
S31508022EACB28007EE102AB8EE477A9FED696AC6EE2B
S31508022EBC076A664B9B6BC3F3080307EE103AB8EE28
S31508022ECC477A9FED646A67EE867A77EE277AB7EECB
S31508022EDC007A77EE877A66EEA76A61E05B4B1B6827
S31508022EEC13F0200F23D0594C2168C1F3C1015A4B58
S31508022EFCCB4007EE103AB8EE477A06EE902AB8EEB1
S31508022F0C666AC7EE066AA36BC3F3080307EE103AA2
S31508022F1CB8EE477A9FED4F6A67EE867A77EE277A8E
S31508022F2CB7EE007A77EE877A66EEA76A38E007EE8E
S31508022F3C102AB8EE477A9FED496AC6EE076A434BE2
S31508022F4C9B6BC3F3080307EE103AB8EE477A9FED6C
S31508022F5C416A67EE867A77EE277AB7EE007A77EECB
S31508022F6C877A66EEA76A1BE007EE102AB8EE477A4E
S31508022F7C9FED376AC6EE076A344B9B6BC3F308039D
S31508022F8C07EE103AB8EE477A9FED326A67EE867A02
S31508022F9C77EE277AB7EE007A77EE877A66EEA76A25
S31508022FAC2A4A936BC3F3462307EE103AB8EE477ACE
S31508022FBCB7EE006A37EE067AC6EE877AFCEEE77A41
S31508022FCCC0ED007A936BC3F3064307EE103AB8EEDC
S31508022FDC477A37EE067AC6EE877AFCEEE77AC0EDC2
S31508022FEC017A936BC3F3066307EE903AF8EE677AA7
S31508022FFC77EE867A86EEA77ABCEEC77A80ED027AE7
S3150802300C5DF8044B704707EE102AB8EE477A9FED27
S3150802301C146AC6EE076A0D4B9B6BC3F3080307EEDD
S3150802302C103AB8EE477A9FED0B6A67EE867A77EE18
S3150802303C277AB7EE007A77EE877A66EEA76AAFE753
S3150802304C0023036043608360DAE700BF004402583A
S3150802305C0024744A000000390090D0030024744CF2
S3150802306C0024F44A10B478498C6A8A6AC2F3055267
S3150802307CCB6AC3F30023496CC1F3CC0103FB01F3FE
S3150802308C002A00F0DB8004F0030407EE903AF8EE0F
S3150802309C677A012C66D0FCB1022C00F0B28007EEDE
S315080230AC102AB8EE477A9FED696AC6EE076A664B2E
S315080230BC1B6CC3F3080307EE103AB8EE477A9FED7A
S315080230CC646A67EE867A77EE277AB7EE007A77EE37
S315080230DC877A66EEA76A61E05B4B1B6813F0200FD2
S315080230EC23D0594C2168C1F3C1015A4BCB4007EE88
S315080230FC103AB8EE477A06EE902AB8EE666AC7EE2A
S3150802310C066A236CC3F3080307EE103AB8EE477A3D
S3150802311C9FED4F6A67EE867A77EE277AB7EE007AD4
S3150802312C77EE877A66EEA76A38E007EE102AB8EECB
S3150802313C477A9FED496AC6EE076A434B1B6CC3F383
S3150802314C080307EE103AB8EE477A9FED416A67EE26
S3150802315C867A77EE277AB7EE007A77EE877A66EE74
S3150802316CA76A1BE007EE102AB8EE477A9FED376A74
S3150802317CC6EE076A344B1B6CC3F3080307EE103A08
S3150802318CB8EE477A9FED326A67EE867A77EE277A39
S3150802319CB7EE007A77EE877A66EEA76A2A4A136C36
S315080231ACC3F3462307EE103AB8EE477AB7EE006A2F
S315080231BC37EE067AC6EE877AFCEEE77AC0ED007A27
S315080231CC136CC3F3064307EE103AB8EE477A37EE9A
S315080231DC067AC6EE877AFCEEE77AC0ED017A136CAC
S315080231ECC3F3066307EE903AF8EE677A77EE867AB9
S315080231FC86EEA77ABCEEC77A80ED027A5DF8044BA6
S3150802320C704707EE102AB8EE477A9FED146AC6EE97
S3150802321C076A0D4B1B6CC3F3080307EE103AB8EE9C
S3150802322C477A9FED0B6A67EE867A77EE277AB7EEC0
S3150802323C007A77EE877A66EEA76AAFE70023036011
S3150802324C43608360DAE700BF004402580024744ADC
S3150802325C000000390090D0030024744C0024F44A70
S3150802326C2DE9F04387B00446016883680269134363
S3150802327C42691343C2691343426E13430868884A68
S3150802328C02401A430A602268536823F44053E168E1
S3150802329C0B435360A1692268824B9A4201D0236A76
S315080232AC19439068804B03400B4393602268D36A98
S315080232BC23F00F03616A0B43D36223687B4A93425A
S315080232CC1FD07B4A934259D07A4A934270D07A4A93
S315080232DC934200F08780794A934200F09D80784A9F
S315080232EC934200F0B380774A934200F0F180764A13
S315080232FC934200F004816B4A934200F017818022B4
S3150802330C2DE1724A526D02F03802282A34D8DFE8C7
S3150802331C12F0290033003300330033003300330034
S3150802332C33002501330033003300330033003300F6
S3150802333C33002B00330033003300330033003300E1
S3150802334C33002D00330033003300330033003300CF
S3150802335C33002F00330033003300330033003300BD
S3150802336C330031000122FAE00822F8E01022F6E0D6
S3150802337C2022F4E04022F2E08022F0E0534A526D19
S3150802338C02F00702052A11D8DFE812F00600370107
S3150802339C08000A000C000E000022E0E00822DEE01B
S315080233AC1022DCE02022DAE04022D8E08022D6E0A5
S315080233BC464A526D02F00702052A11D8DFE812F0C6
S315080233CC06001F0108000A000C000E000022C6E0C7
S315080233DC0822C4E01022C2E02022C0E04022BEE04D
S315080233EC8022BCE0394A526D02F00702052A11D82E
S315080233FCDFE812F00600070108000A000C000E00AE
S3150802340C0022ACE00822AAE01022A8E02022A6E0BC
S3150802341C4022A4E08022A2E02C4A526D02F0070256
S3150802342C052A11D8DFE812F00600EF0008000A0098
S3150802343C0C000E00002292E0082290E010228EE088
S3150802344C20228CE040228AE0802288E01F4A526DB4
S3150802345C02F03802282A20D8DFE802F0151F1F1FAF
S3150802346C1F1F1F1FD71F1F1F1F1F1F1F171F1F1FA0
S3150802347C1F1F1F1F191F1F1F1F1F1F1F1B1F1F1F4A
S3150802348C1F1F1F1F1D00012269E0082267E0102278
S3150802349C65E0202263E0402261E080225FE000BF03
S315080234ACF369FFCF000C0058FFF4FF11001001401E
S315080234BC0044004000480040004C004000500040C8
S315080234CC0014014000780040007C00400044025879
S315080234DC824A526D02F00702052A0ED8DFE802F07C
S315080234EC03970507090B002239E0082237E0102258
S315080234FC35E0202233E0402231E080222FE0774A61
S3150802350C526D02F00702052A0ED8DFE802F0038292
S3150802351C0507090B002222E0082220E010221EE0F1
S3150802352C20221CE040221AE0802218E002F50E3214
S3150802353C926D02F00702052A0ED8DFE802F0036C38
S3150802354C0507090B02220AE0082208E0102206E007
S3150802355C202204E0402202E0802200E00422604994
S3150802356C8B425AD0E369B3F5004F00F0C380402A68
S3150802357C00F27981DFE812F027014B017701770116
S3150802358C4E017701770177015301770177017701AC
S3150802359C770177017701770158017701770177016E
S315080235AC770177017701770177017701770177013F
S315080235BC7701770177017701250177017701770181
S315080235CC770177017701770177017701770177011F
S315080235DC770177017701770177017701770177010F
S315080235EC77017701770177017701770177017701FF
S315080235FC770177017701770164010422AFE7042288
S3150802360CADE70422ABE70422A9E70422A7E70422C2
S3150802361CA5E70422A3E70422A1E7082A48D007D97A
S3150802362C202A0ED0402A54D0102A46D00120E3E094
S3150802363C022A08D0042AF9D103A8FFF715FC049824
S3150802364C03E0284804E0FFF7FDFB002800F0FD80A4
S3150802365C626A254B33F81220B0FBF2F3656805EB68
S3150802366C4501994200F2F380B3EB053F00F2F18073
S3150802367C4FF0000892B200234146FCF729FE0F02CE
S3150802368C47EA1067060268082A46434616EB0008FC
S3150802369C47F1000940464946FCF71AFEA0F5407266
S315080236AC124B9A4200F2D7802368D8600020A3E016
S315080236BC6846FFF7D7FC0198C7E7084B1B6813F057
S315080236CC200F09D0054B1B68C3F3C1030848D84021
S315080236DCBBE74FF40040BBE70548B9E7004402587C
S315080236EC000C005800093D001C3D0208FFFC0F00A7
S315080236FC0090D003402A00F2B080DFE802F023449F
S3150802370CAEAE47AEAEAE4CAEAEAEAEAEAEAE51AEE3
S3150802371CAEAEAEAEAEAEAEAEAEAEAEAEAEAE21AE3A
S3150802372CAEAEAEAEAEAEAEAEAEAEAEAEAEAEAEAE9D
S3150802373CAEAEAEAEAEAEAEAEAEAEAEAEAEAE5D008C
S3150802374C4C4804E0FEF7B2FD002800F08880626A55
S3150802375C494B33F81230B0FBF3F06268530803EBAB
S3150802376C4003B3FBF2F39BB2A3F110014FF6EF72CF
S3150802377C914276D823F00F02C3F34203134322680D
S3150802378CD360002038E0FEF7A3FDDDE703A8FFF7B8
S3150802379C6BFB0498D8E76846FFF764FC0198D3E7F5
S315080237AC364B1B6813F0200F09D0344B1B68C3F336
S315080237BCC1033348D840C7E74FF40040C7E730483F
S315080237CCC5E72C4803E0FEF771FD00284DD0626A66
S315080237DC294B33F81230B0FBF3F0636800EB530055
S315080237ECB0FBF3F080B2A0F110024FF6EF739A42D7
S315080237FC3DD82368D86000200123A4F86A30A4F8BF
S3150802380C68300023E366236707B0BDE8F083FEF74A
S3150802381C5FFDDAE703A8FFF727FB0498D5E76846A6
S3150802382CFFF720FC0198D0E7144B1B6813F0200F06
S3150802383C09D0124B1B68C3F3C1031148D840C4E71D
S3150802384C4FF40040C3E70E48C1E70020D4E7012035
S3150802385CD2E70120D0E70120CEE70120CCE70020F1
S3150802386CCAE70120C8E70120C6E70020C4E7012001
S3150802387CC2E700BF00093D001C3D0208004402587D
S3150802388C0090D003836A13F0010F06D002685368BE
S3150802389C23F40033C16A0B435360836A13F0020F95
S315080238AC06D00268536823F48033016B0B435360CA
S315080238BC836A13F0040F06D00268536823F4802334
S315080238CC416B0B435360836A13F0080F06D00268E8
S315080238DC536823F40043816B0B435360836A13F0DA
S315080238EC100F06D00268936823F48053C16B0B43FE
S315080238FC9360836A13F0200F06D00268936823F448
S3150802390C0053016C0B439360836A13F0400F0AD081
S3150802391C0268536823F48013416C0B435360436C5F
S3150802392CB3F5801F0BD0836A13F0800F06D002689A
S3150802393C536823F40023C16C0B4353607047026827
S3150802394C536823F4C003816C0B435360EBE72DE9F0
S3150802395CF04104460F4616469846069D2368DB69CF
S3150802396C37EA03030CBF01230023B3423FD1B5F157
S3150802397CFF3FF3D0FDF7F4F9A0EB0800A84222D8D2
S3150802398C0DB323681A6812F0040FE7D0DA6912F439
S3150802399C006FE3D04FF400621A622268136823F4AC
S315080239ACD07313602268936823F001039360202373
S315080239BCC4F88030C4F88430C4F88830002384F8FC
S315080239CC7C30032014E02268136823F4D073136046
S315080239DC2268936823F0010393602023C4F880308D
S315080239ECC4F88430002384F87C30032000E00020DD
S315080239FCBDE8F0812DE9F04383B01E46D0F8843039
S31508023A0C202B40F0838004460D469046B2FA82F388
S31508023A1C5B09002908BF0123002B7BD190F87C3067
S31508023A2C012B79D0012380F87C300023C0F888302A
S31508023A3C2223C0F88430FDF793F90746A4F85C8074
S31508023A4CA4F85E80A368B3F5805F06D0A3B9226991
S31508023A5C72B9FF22A4F8602014E0226922B940F256
S31508023A6CFF12A4F860200DE0FF22A4F8602009E0FA
S31508023A7C7F22A4F8602005E0B3F1805F0DD0002206
S31508023A8CA4F86020B4F86080B3F5805F0FD04FF0CD
S31508023A9C0009002384F87C301DE022691AB97F22BA
S31508023AACA4F86020EEE73F22A4F86020EAE723692F
S31508023ABC13B14FF00009ECE7A9460025E9E723689C
S31508023ACC5B6A08EA030329F8023BB4F85E30013B49
S31508023ADC9BB2A4F85E30B4F85E309BB28BB10096FA
S31508023AEC3B46002220212046FFF731FFB0B9002DB4
S31508023AFCE5D023685A6A5FFA88F3134005F8013B46
S31508023B0CE3E72023C4F88430002000E0022003B047
S31508023B1CBDE8F0830120FAE70220F8E70320F6E76E
S31508023B2C30B583B004460023C0F88830FDF718F97F
S31508023B3C054623681B6813F0080F0ED123681B6809
S31508023B4C13F0040F17D12023C4F88030C4F884303C
S31508023B5C002084F87C0003B030BD6FF07E430093DE
S31508023B6C034600224FF400112046FFF7F0FE002808
S31508023B7CE4D00320EFE76FF07E4300932B46002236
S31508023B8C4FF480012046FFF7E2FE0028DBD0032023
S31508023B9CE1E778B310B50446D0F880300BB324238A
S31508023BACC4F880302268136823F001031360204698
S31508023BBCFFF756FB012813D0A36ABBB922685368D0
S31508023BCC23F4904353602268936823F02A03936084
S31508023BDC2268136843F0010313602046FFF7A0FF1F
S31508023BEC10BD80F87C30FCF77FFFD8E72046FFF73C
S31508023BFC49FEE3E70120704770B50D4E0D4CA41B28
S31508023C0CA4100025A54209D10B4E0C4C00F02CF839
S31508023C1CA41BA4100025A54205D170BD56F8253063
S31508023C2C98470135EEE756F8253098470135F2E7FD
S31508023C3C3C3D02083C3D02083C3D0208403D020858
S31508023C4C10B5431E0A44914200D110BD11F8014B1E
S31508023C5C03F8014FF7E702440346934200D1704733
S31508023C6C03F8011BF9E70000F8B500BFF8BC08BC5D
S31508023C7C9E467047F8B500BFF8BC08BC9E4670470E
S31508023C8C0000000000000000000000000000000018
S31508023C9C0000000001000000020000000300000002
S31508023CAC04000000000000000500000000000000EF
S31508023CBC00000000000000000600000000000000E2
S31508023CCC00000000000000000700000005020602C2
S31508023CDC060307030803090309040A040B040C0464
S31508023CEC0C050D050E050F050F0610061007100814
S31508023CFC0000000001020304010203040607080976
S31508023D0C0001020304050607080C1014182030409B
S31508023D1C010002000400060008000A000C0010004C
S30D08023D2C20004000800000019E
S30D08023D34D8C5FF7F010000005B
S30908023D3CC1020208A6
S30908023D409D020208C6
S31508023D440090D0030090D003010000001000000088
S70508020C558F
